S01C000064656D6F70726F675F646B5F746D3463313233672E73726563A9
S113200050040020FD290000152A0000152A0000B4
S1132010152A0000152A0000152A0000152A0000C0
S1132020152A0000152A0000152A0000152A0000B0
S1132030152A0000152A0000152A0000AF28000008
S1132040152A0000152A0000152A0000152A000090
S1132050152A0000152A0000152A0000152A000080
S1132060152A0000152A0000152A0000152A000070
S1132070152A0000152A0000152A0000152A000060
S1132260152A0000152A0000152A0000EE11AA55AF
S1132270C0F30721DFF828225118C0B2800050EAC9
S1132280411050F08440012101607047DFF82002C2
S1132290DFF820120160FEE70138FDD17047704776
S11322A070B504007F4805688348066855F40065E6
S11322B035F4800556F400667A4805607E48066069
S11322C015F0010014F0010191F00101C0B20842BF
S11322D01DD074F00100054072480560002E07D53A
S11322E016F07000302809D016F07000702805D060
S11322F0002E08D415F03000302804D14FF480505B
S1132300FFF7CAFF03E05FF40020FFF7C5FF35F4D1
S1132310FE6514F4FE6005436848064068482040A2
S1132320064314F0080056EAC0065E480560624899
S113233006601020FFF7B0FF35F4005514F4005088
S1132340054336F4005614F4005006435648402121
S11323500160002E04D5584806605248056003E029
S11323605048056054480660564805405648204089
S1132370054336F0FC5614F0FC500643600007D5C4
S113238055F4800536F4800650482040064301E0A9
S113239036F0804620050DD44FF4004000E0401E86
S11323A0002803D0414909684906F8D535F4006589
S11323B036F400663B4805603F4806601020FFF78E
S11323C06BFF70BD30B4374801683B480268002A8F
S11323D002D512F0700001E011F03000002808D09E
S11323E0102844D0202844D0302844D0702845D028
S11323F047E0C1F38410364B53F82000354B1340AB
S113240013F1004F03D0002A1BD40B0519D4324B0F
S11324101B68324C2468C4F304256D1C14F01F049B
S1132420641C04FB05F46400B0FBF4F09C05A40DEB
S1132430C3F3892303FB00F39B0A04FB003051F42C
S113244080014B022AD5002A23D553001BD5214BEA
S1132450134013F1004F03D0002A14D4090512D4F9
S11324604000C2F38651491CB0FBF1F016E01C4851
S1132470C4E71C48C2E747F23050BFE74FF40040BE
S1132480BCE700200AE0C2F3C551491CB0FBF1F0DF
S113249004E0C1F3C351491CB0FBF1F030BC7047F8
S11324A000E60F4060E00F4058E00F4050E00F405E
S11324B00CED00E00400FA0570E00F408FFFFF7F91
S11324C030000080FEFF3FF80100C00700004040DC
S11324D0EC2800000008008060E10F4064E10F4038
S11324E00024F40000093D0010B4D30705D510F50D
S11324F080631B68C9B20B4304E010F580631B685A
S1132500C9B28B4310F580642360920705D510F59A
S113251084621268C9B2114305E010F5846212683E
S1132520C9B232EA010110F58460016010BC704741
S113253030B4D40705D510F5A0642468C9B20C439F
S113254004E010F5A0642468C9B28C4310F5A065BA
S11325502C60940704D5D0F80445C9B20C4303E0B9
S1132560D0F80445C9B28C43C0F80445540705D5D6
S113257010F5A1642468C9B20C4304E010F5A16409
S11325802468C9B28C4310F5A1652C60120705D5E7
S113259010F5A3621268C9B20A4304E010F5A362FD
S11325A01268C9B28A4310F5A3642260DA0704D51D
S11325B0D0F80C25C9B20A4303E0D0F80C25C9B2FF
S11325C08A43C0F80C259A0705D510F5A262126853
S11325D0C9B20A4304E010F5A2621268C9B28A4380
S11325E010F5A26422605A0704D5D0F81425C9B2A4
S11325F00A4303E0D0F81425C9B28A43C0F814256D
S11326001A0704D5D0F81C25C9B20A4303E0D0F850
S11326101C25C9B28A43C0F81C25002B05D110F52E
S1132620A5621268C9B2114305E010F5A5621268EB
S1132630C9B232EA010110F5A560016030BC7047EF
S1132640C9B2D2B240F82120704738B504000D0059
S1132650082301222900C9B22000FFF769FF0122E3
S11326602900C9B22000FFF73FFF31BD38B504008F
S11326700D0002222900C9B22000FFF735FF08230C
S113268001222900C9B22000FFF752FF31BD50F8E2
S1132690041B61B150F8042BD30744BFA9F1010313
S11326A09A18002342F8043B091FFAD1EFE7704758
S11326B080B5FFF7EBFD01BD80B52A48FFF7D8FDD3
S11326C02948FFF7D5FD03215FF04020FFF7CEFF37
S11326D0FFF778FE60234FF461420100234800F0C5
S11326E04DF801BD80B52248007800280BD121485F
S11326F000F02BF8012827D11D48012101701E4844
S11327000021017020E01C4800781A494018401C40
S113271000F01BF8012817D117480078401C16490F
S11327200870154800781349097888420CD110487C
S1132730002101700F484078FF2805D10D488078AA
S1132740002801D1FFF7B4FF01BD10B5040007480C
S113275000F056F810F1010F02D02070012000E0C3
S1132760002010BD001800F0000800F000C0004078
S11327704D000020000000204C000020F8B50400AB
S11327800F0016001D00200000F02BF8B7EB061F09
S113279005D2206B50F020002063760803E0206B04
S11327A030F020002063F800B0FBF6F0401C400835
S11327B0810961624021B0FBF1F202FB1102A262C5
S11327C0E5620020A061200000F001F8F1BDC16ABB
S11327D051F01001C162016B40F2013211430163F7
S11327E0704781690907FCD4C16A31F01001C162E4
S11327F0016B024A1140016370470000FEFCFFFFB9
S11328008169C90601D4006801E05FF0FF307047B8
S113281080B51748FFF72CFD04211648FFF715FF74
S1132820002204211348FFF70BFF01BD10B500F08F
S11328303BF8040010480068201AB0F5FA7F16D35C
S11328400E480078002808D10C48012101700422A8
S113285004210848FFF7F4FE07E00848002101704E
S1132860002204210348FFF7EBFE0348046010BD77
S1132870060800F000600240440000204E000020E2
S113288080B5FFF79FFD4FF47A71B0FBF1F000F0D3
S113289025F800F015F800F01AF8002000F001F80F
S11328A001BD064908607047044800687047034842
S11328B00068401C0149086070470000480000207F
S11328C00848006850F0050006490860704705484C
S11328D0006850F00200034908607047401E024936
S11328E00860704710E000E014E000E040420F0090
S11328F000201C0080841E0000802500999E360064
S11329000040380000093D0000803E0000004B00FC
S1132910404B4C0000204E00808D5B0000C05D00E9
S11329200080700000127A0000007D0080969800FC
S1132930001BB7000080BB00C0E8CE00647ADA0058
S11329400024F4000000FA0080A81201002D3101D7
S113295000366E0140787D0180B500F007F8FFF77E
S1132960ABFEFFF763FFFFF7BDFEFAE780B500F0AB
S11329700DF80548FFF794FCFFF74AFFFFF780FFC7
S113298000F00EF801BD00004005C00103480068D6
S113299050F04040014908607047000034EF00E007
S11329A080B500F001F801BD80B500F007F80028FB
S11329B001D0012000E00020C0B202BDEFF310807E
S11329C062B6704710B5074979441831064C7C4407
S11329D0163404E00A68081D511888470146A142CC
S11329E0F8D110BD0800000014000000A3FCFFFF94
S11329F050000000000000200000000080B50448E2
S1132A00006850F470000249086000F005F801BD48
S1132A1088ED00E0FEE70000034B9D46C046C0463B
S1132A2000F004F800F010F8500400204EF688512D
S1132A30CEF20001086840F4700008604FF00070A6
S1132A40E1EE100A7047000000F009F8002801D0F8
S1132A50FFF7B8FF0020FFF77FFF00F002F8012026
S1132A60704700F001B800000746384600F002F84D
S1132A70FBE7000080B5C046C046024A110018209A
S10B2A80ABBEFBE726000200D7
S9032A19B9
